S01A000064656D6F70726F675F73746D3332663230372E7372656396
S3150800800000000220D19C0008219D0008219D00083F
S31508008010219D0008219D0008219D00080000000000
S31508008020000000000000000000000000219D00087C
S31508008030219D000800000000219D0008599D0008A8
S31508008040219D0008219D0008219D0008219D00080A
S31508008050219D0008219D0008219D0008219D0008FA
S31508008060219D0008219D0008219D0008219D0008EA
S31508008070219D0008219D0008219D0008219D0008DA
S31508008080219D0008219D0008219D0008219D0008CA
S31508008090219D0008219D0008219D0008219D0008BA
S315080080A0219D0008219D0008219D0008219D0008AA
S315080080B0219D0008219D0008219D0008219D00089A
S315080080C0219D0008219D0008219D0008219D00088A
S315080080D0219D0008219D0008219D0008219D00087A
S315080080E0219D0008219D0008219D0008219D00086A
S315080080F0219D0008219D0008219D0008219D00085A
S31508008100219D0008219D0008219D0008219D000849
S31508008110219D0008219D0008219D0008219D000839
S31508008120219D0008219D0008219D0008219D000829
S31508008130219D0008219D0008219D0008219D000819
S31508008140219D0008219D0008219D0008219D000809
S31508008150219D0008219D0008219D0008219D0008F9
S31508008160219D0008219D0008219D0008219D0008E9
S31508008170219D0008219D0008219D0008000000009F
S30D08008180219D0008EE11AA5525
S3150800818810B5054C237833B9044B13B10448AFF33B
S3150800819800800123237010BD0400002000000000A1
S315080081A8AC9D000808B5034B1BB103490348AFF358
S315080081B8008008BD0000000008000020AC9D0008EB
S315080081C853B94AB9002908BF00281CBF4FF0FF3128
S315080081D84FF0FF3000F07AB9ADF1080C6DE904CE1E
S315080081E800F006F8DDF804E0DDE9022304B070477C
S315080081F82DE9F0478C460E460446089D002B50D1BB
S315080082088A4217466CD9B2FA82FEBEF1000F0BD025
S31508008218CEF1200C01FA0EF620FA0CFC02FA0EF73B
S315080082284CEA060C00FA0EF43A0CBCFBF2F9BBB29F
S3150800823802FB19CC09FB03FA4FEA144848EA0C462C
S31508008248B2450AD9F61909F1FF3180F02581B245F8
S3150800825840F22281A9F102093E44A6EB0A06B6FBBA
S31508008268F2F002FB106600FB03F3A4B244EA0644E4
S31508008278A34209D9E41900F1FF3280F00B81A34221
S3150800828840F2088102383C440021E41A40EA0940D1
S31508008298002D62D0002324FA0EF42C606B60BDE82A
S315080082A8F0878B4207D9002D55D0002185E8410073
S315080082B80846BDE8F087B3FA83F1002940F08F80B5
S315080082C8B34202D3824200F2FC80841A66EB0306A4
S315080082D80120B446002D40D085E81010BDE8F08787
S315080082E812B90127B7FBF2F7B7FA87FEBEF1000FF6
S315080082F835D10121F61B4FEA174C1FFA87F8B6FB4A
S31508008308FCF20CFB126608FB02F0230C43EA06464D
S31508008318B04207D9F61902F1FF3302D2B04200F289
S31508008328D2801A46361AB6FBFCF00CFB106608FB18
S3150800833800F8A3B243EA0644A04507D9E41900F1B0
S31508008348FF3302D2A04500F2B9801846A4EB080408
S3150800835840EA02409CE729462846BDE8F08707FA1E
S315080083680EF7CEF1200326FA03F24FEA174CB2FBB2
S31508008378FCF11FFA87F80CFB112206FA0EF620FA0A
S3150800838803F301FB08F933431E0C46EA0246B145D6
S3150800839800FA0EF409D9F61901F1FF3280F08C803B
S315080083A8B14540F2898002393E44A6EB0906B6FB78
S315080083B8FCF00CFB106200FB08F99EB246EA02467E
S315080083C8B14507D9F61900F1FF3371D2B1456FD90E
S315080083D802383E44A6EB090640EA01418FE7C1F197
S315080083E8200722FA07F88B4048EA030326FA07F417
S315080083F84FEA134EB4FBFEF91FFA83FC0EFB194429
S315080084088E4020FA07F809FB0CFA48EA06084FEAEC
S31508008418184646EA0444A24502FA01F200FA01F6A9
S3150800842808D9E41809F1FF3044D2A24542D9A9F17E
S3150800843802091C44A4EB0A04B4FBFEF00EFB104424
S3150800844800FB0CFC1FFA88F848EA0444A44507D937
S31508008458E41800F1FF3E29D2A44527D902381C445E
S3150800846840EA0940A0FB0289A4EB0C0CCC45C2469D
S31508008478CE4615D312D055B1B6EB0A036CEB0E06E9
S3150800848806FA07F7CB401F43CE402F606E600021DF
S31508008498BDE8F0871046F7E68946DEE64645EAD29D
S315080084A8B8EB020A69EB030E0138E4E77046D7E72A
S315080084B818468FE78146BDE7114676E702383C44F9
S315080084C844E7084606E7023A3E442BE7704700BFEA
S315080084D808B50848084B03604FF461434360002316
S315080084E88360C360036183610C23436101F045FA25
S315080084F808BD00BF88000020004800402DE9F0416B
S3150800850804460D461746984601F036F8154BA3FB60
S3150800851800308009002201E00132D2B2112A1ED8A1
S31508008528114B13F8121003EB420393F801E001EB21
S315080085380E0303FB0443B0FBF3FC03FB1C06002EE7
S31508008548EAD11FFA8CF32B80013B9BB2B3F5806FF7
S31508008558E2D2397088F800E00120BDE8F0810020F1
S31508008568BDE8F081D34D6210C49D000870B58CB083
S315080085780025ADF82E508DF82D500CAB03F8045D88
S315080085880DF12D020DF12E014FF4FA70FFF7B6FF23
S315080085981D4C1E4E266025631D4B6363A561E56168
S315080085A825626562A562E562A560E5609DF82D30DD
S315080085B8013B1B0423619DF82C30013B1B056361B5
S315080085C8BDF82E306360204600F0B9F92368B34237
S315080085D818D00E23069300230793012208924CF617
S315080085E8E041019102934FF6E07103910421049149
S315080085F8059309920E230A936944034800F014F96F
S315080086080CB070BD0695E6E720000020006400401F
S315080086186400002008B5002301220146034801F03A
S31508008628DBF908B1002008BD012008BD8800002034
S3150800863808B5FFF74DFFFFF799FF08BDBFF34F8F42
S315080086480549CA6802F4E062044B1343CB60BFF3DA
S315080086584F8F00BFFDE700BF00ED00E00400FA05F4
S3150800866808B5214B1B78B3B92048FFF7D3FF012873
S3150800867800D008BD1D4B1B78013BDBB23F2BF8D851
S3150800868801F062FB1A4B18600122174B1A70002278
S31508008698184B1A7008BD174B1B7801331348184432
S315080086A8FFF7B8FF01280AD001F04EFB104B1B68EC
S315080086B864339842DDD900220B4B1A70D9E70D4A64
S315080086C813780133DBB21370084A12789342D0D173
S315080086D80021054A1170054A5278FF2AC9D1022B8A
S315080086E8C7D1FFF7ABFF00BF09010020C80000206B
S315080086F80C0100200A01002008B5002211460E4880
S3150800870800F0DDF940B90C4B5B6B196840F26762FB
S31508008718914202D0002232B908BD9A680AB10022ED
S31508008728F9E70122F7E71A7DFF2AF5D11B69022B1B
S31508008738F2D1FFF783FF00BF2000002008B5FFF736
S315080087488FFFFFF7D9FF08BD08B500224FF48071DF
S31508008758014800F059FC08BD0014024010B501F0A4
S31508008768F3FA0F4B1B68C31AB3F5FA7F0DD3044601
S315080087780C4B1B7853B901220A4B1A704FF48071B7
S31508008788094800F041FC064B1C6010BD0022054B49
S315080087981A704FF48071044800F036FCF3E700BFFE
S315080087A814010020100100200014024010B50446E8
S315080087B8074B1868074BA3FB0030800900F00CFB31
S315080087C8002221464FF0FF3000F0D4FA002010BDF1
S315080087D800000020D34D621008B50B4B1A6842F406
S315080087E800721A601A6842F480621A601A6842F4BB
S315080087F880721A60032000F0ABFA0020FFF7D6FF54
S3150800880801F0C8F9002008BD003C0240024A136876
S3150800881801331360704700BF18010020014B186820
S31508008828704700BF1801002070B44B6901229A40AE
S31508008838414BD3F8000240F00100C3F80002D3F810
S31508008848000220F47C50C3F80002D3F800024C6AF0
S3150800885840EA0420C3F80002D3F81C42D043044077
S31508008868C3F81C42CB69B3B9334BD3F80C4204405E
S31508008878C3F80C424C69CE688D8845EA06454834E3
S3150800888843F834504D698E680C8844EA06444835DE
S3150800889803EBC5035C60CB69012B20D08B69002BE1
S315080088A835D1254CD4F804320340C4F804320B6990
S315080088B82BB9214BD3F814422040C3F814020B698C
S315080088C8012B2BD00B6A012B2FD01B4AD2F800326A
S315080088D823F00103C2F80032002070BC7047164B1B
S315080088E8D3F80C421443C3F80C424C690E688D88B9
S315080088F845EA0645483443F834504D698E688C89EC
S3150800890844EA0644483503EBC5035C60C6E70A4CE7
S31508008918D4F804321343C4F80432C8E70648D0F832
S3150800892814321343C0F81432CCE7034BD3F81C129D
S315080089380A43C3F81C22C8E70064004070470028A9
S3150800894800F0BB8038B5044690F83C3003B30223E0
S3150800895884F83C302268136823F0020313602268FF
S31508008968136843F001031360FFF758FF05462368A9
S315080089785A6812F0010F10D1FFF750FF401B0A285A
S31508008988F5D9032084F83C00002384F83D3038BD27
S3150800899880F83D30FFF7D2FFD9E75A6812F0010F81
S315080089A87CD0A269012A50D01A6822F080021A607F
S315080089B8E369012B4ED02268136823F0400313603D
S315080089C8236A012B4CD02268136823F0200313600E
S315080089D8636A012B4AD02268136823F010031360D0
S315080089E8A36A012B48D02268136823F0080313608A
S315080089F8E36A012B46D02268136823F00403136040
S31508008A082168A368E268134322691343626913431A
S31508008A186268013A1343CB612268136823F001039D
S31508008A281360FFF7FBFE054623685A6812F0010F24
S31508008A382ED0FFF7F3FE401B0A28F5D9032084F841
S31508008A483C00002384F83D3038BD1A6842F080029D
S31508008A581A60ADE72268136843F040031360AFE76E
S31508008A682268136843F020031360B1E72268136885
S31508008A7843F010031360B3E72268136843F008034A
S31508008A881360B5E72268136843F004031360B7E771
S31508008A985B6813F0010F08D0002300E0002333B900
S31508008AA8042384F83C30012038BD0123F7E7002069
S31508008AB82064012384F83C3038BD01207047F8B596
S31508008AC80D46B9B990F83C30DBB2222B00F02F815D
S31508008AD890F83C30DBB2422B00F02B8190F83C3002
S31508008AE8DBB2622B00F0278190F83C30DBB2722BA0
S31508008AF800F02381012D15D090F83D30012B00F0A8
S31508008B082481012380F83D30B5BB90F83C30DBB2B0
S31508008B18322B29D0522B2BD0122B1CD0222380F88B
S31508008B283C301BE090F83C30DBB2322B00F0078172
S31508008B3890F83C30DBB2522B00F0038190F83C30B9
S31508008B48DBB2622B00F0FF8090F83C30DBB2722B68
S31508008B58D2D10220F8BD422380F83C301646044696
S31508008B68FFF75CFE074638E0622380F83C30F5E7F5
S31508008B78722380F83C30F1E790F83C30DBB2222BC0
S31508008B880BD0422B0DD0122B03D0322380F83C3061
S31508008B98E4E7522380F83C30E0E7622380F83C306B
S31508008BA8DCE7722380F83C30D8E726B1FFF736FEB3
S31508008BB8C01B864211D2032084F83C00002384F89F
S31508008BC83D30F8BD23681B6913F0030F0CBF01235A
S31508008BD8002363B1B6F1FF3FE7D1002DF2D1236830
S31508008BE8DB6813F0030F0CBF01230023F1E7002D00
S31508008BF867D1636B216805F11B0212018A5802F0D6
S31508008C0804029A60002A5ED1216805F11B02120146
S31508008C188A58520D1A60216805F11B0212018958F3
S31508008C2801F00201D96021681144496801F00F0171
S31508008C38196121680A445268C2F30722DA611D627B
S31508008C4821682A011144D1F8B81119752168114407
S31508008C58D1F8B811090A597521681144D1F8B8111B
S31508008C68090C997521681144D1F8B811090ED975F6
S31508008C7821681144D1F8BC11197621681144D1F834
S31508008C88BC11090A597621681144D1F8BC11090C96
S31508008C98997621680A44D2F8BC21120EDA76D5B933
S31508008CA823682022DA604DBB94F83C30DBB2622B8D
S31508008CB81CD0722B1ED0422B11D0012384F83C30CD
S31508008CC810E0A36B96E7216805F11B0212018A5882
S31508008CD8D2085A609FE7236820221A61E3E712231D
S31508008CE884F83C30002084F83D00F8BD322384F827
S31508008CF83C30F7E7522384F83C30F3E794F83C30E5
S31508008D08DBB2622B0BD0722B0DD0522B03D001236A
S31508008D1884F83C30E6E7122384F83C30E2E722235D
S31508008D2884F83C30DEE7422384F83C30DAE7022050
S31508008D38F8BD0220F8BD0220F8BD0220F8BD0220C1
S31508008D48F8BD0220F8BD0220F8BD0220F8BD0000D3
S31508008D58074AD36823F4E0631B041B0C000200F4DB
S31508008D68E060184340F0BF6040F40030D0607047B8
S31508008D7800ED00E030B4164BDB68C3F30223C3F1F9
S31508008D880704042C28BF04241D1D062D17D9033BE8
S31508008D98012505FA04F4013C2140994005FA03F334
S31508008DA8013B1340194300280BDB0901C9B200F13E
S31508008DB8604000F5614080F8001330BC7047002316
S31508008DC8E6E700F00F000901C9B2024B1954F4E7A7
S31508008DD800ED00E014ED00E00138B0F1807F0AD21A
S31508008DE8064B5860F021064A82F82310002098603E
S31508008DF807221A6070470120704700BF10E000E09C
S31508008E0800ED00E0042805D0054A136823F004039A
S31508008E1813607047024A136843F0040313607047E7
S31508008E2810E000E0704708B5FFF7FCFF08BD000032
S31508008E38F0B583B000244BE04FEAD40E0EF1080EC5
S31508008E4850F82E2004F00706B6000F27B74022EA86
S31508008E5807020F6907FA06F6324340F82E2046E05D
S31508008E68082600E0002606FA0EF632430233614E5B
S31508008E7846F82320604B1A68EB4302EA03064F6854
S31508008E8817F4803F01D045EA02065B4A1660526825
S31508008E9803EA02064F6817F4003F01D045EA0206BE
S31508008EA8554A5660926803EA02064F6817F4801F07
S31508008EB801D045EA0206504A9660D26813404E68C1
S31508008EC816F4001F01D045EA02034B4AD360013461
S31508008ED80F2C00F28C800123A3400A6803EA0205D6
S31508008EE8AB42F4D14A68022AA6D0122AA4D0066848
S31508008EF84FEA440E032202FA0EF2D24316404F688E
S31508008F0807F0030707FA0EF73E4306604E68771E12
S31508008F18012F03D9112E01D0122E0FD186681640BB
S31508008F28CF6807FA0EF73E438660466826EA0303C3
S31508008F384E68C6F30016A64033434360C3681A4012
S31508008F488B6803FA0EF31A43C2604B6813F0805F06
S31508008F58BDD000230193294B5A6C42F480425A64C7
S31508008F685B6C03F480430193019BA3089E1C214A6A
S31508008F7852F8262004F003064FEA860E0F2606FA4C
S31508008F880EF622EA06021E4FB8423FF46BAF1D4E94
S31508008F98B0421ED006F58066B0421CD006F580663B
S31508008FA8B0421AD006F58066B04218D006F5806633
S31508008FB8B04216D006F58066B04214D006F580662B
S31508008FC8B04212D006F58066B0423FF449AF09268A
S31508008FD849E7012647E7022645E7032643E7042625
S31508008FE841E705263FE706263DE707263BE703B0A0
S31508008FF8F0BD00BF00380140003C0140003802407F
S31508009008000002400004024012B909048161704751
S3150800901881617047002800F0978130B583B004460F
S31508009028036813F0010F2ED0A34B9B6803F00C03BB
S31508009038042B1FD0A04B9B6803F00C03082B14D0F5
S3150800904822799E4B1A706368002B40D0FFF7E6FB1F
S315080090580546994B1B6813F4003F14D1FFF7DEFB4E
S31508009068401B6428F5D9032073E1934B5B6813F416
S31508009078800FE5D0904B1B6813F4003F03D0636854
S31508009088002B00F06381236813F0020F4BD08A4B3C
S315080090989B6813F00C0F2ED0874B9B6803F00C03C4
S315080090A8082B23D0E368002B64D00122844B1A606E
S315080090B8FFF7B4FB0546804B1B6813F0020F4AD12D
S315080090C8FFF7ACFB401B0228F5D9032041E1FFF75F
S315080090D8A5FB0546784B1B6813F4003FD3D0FFF76A
S315080090E89DFB401B6428F5D9032032E1724B5B6867
S315080090F813F4800FD6D1704B1B6813F0020F04D0F7
S31508009108E368012B01D0012023E16B48036823F0AB
S31508009118F8032169F82292FAA2F2B2FA82F201FA5F
S3150800912802F213430360236813F0080F46D06369F5
S3150800913893B30122634B1A60FFF770FB05465E4B33
S315080091485B6F13F0020F39D1FFF768FB401B022843
S31508009158F5D90320FDE05848036823F0F803216988
S31508009168F82292FAA2F2B2FA82F201FA02F213434A
S315080091780360D8E70022524B1A60FFF74FFB0546F3
S315080091884D4B1B6813F0020FCDD0FFF747FB401B6A
S315080091980228F5D90320DCE000224A4B1A60FFF7BB
S315080091A83DFB0546444B5B6F13F0020F06D0FFF7ED
S315080091B835FB401B0228F5D90320CAE0236813F0BB
S315080091C8040F1FD1A369002B00F0C2803A4A92689F
S315080091D802F00C02082A00F0BE80022B59D00022A1
S315080091E8394B1A60FFF71AFB0446334B1B6813F012
S315080091F8007F00F0A780FFF711FB001B6428F4D94D
S315080092080320A6E0002301932B4B1A6C42F08052E8
S315080092181A641B6C03F080530193019B2B4A13684D
S3150800922843F480731360FFF7F9FA0546274B1B6862
S3150800923813F4807F06D1FFF7F1FA401B0228F5D907
S31508009248032086E0227A224B1A70A36883B1FFF7B7
S31508009258E5FA0546184B1B6F13F0020FB2D1FFF754
S31508009268DDFA401B41F288339842F3D9032070E0AF
S31508009278FFF7D4FA0546104B1B6F13F0020FA1D05F
S31508009288FFF7CCFA401B41F288339842F3D90320FA
S315080092985FE000220C4B1A60FFF7C0FA0546064B3A
S315080092A81B6813F0007F15D0FFF7B8FA401B64282F
S315080092B8F5D903204DE000BF0038024002380240C5
S315080092C800004742800E474260004742007000404F
S315080092D870380240E369226A1343616A47F6C07226
S315080092E892FAA2F2B2FA82F201FA02F21343A26AD7
S315080092F85208013A4FF4403191FAA1F1B1FA81F1D5
S315080093088A401343E16A4FF0706292FAA2F2B2FAFF
S3150800931882F201FA02F21343104A53600122104BF3
S315080093281A60FFF77BFA04460C4B1B6813F0007F9C
S3150800933806D1FFF773FA001B6428F5D9032008E05D
S31508009348002006E0002004E001207047012000E024
S31508009358002003B030BD0120FBE700BF00380240FB
S3150800936860004742F8B5254B9B6803F00C03042BAD
S3150800937841D0082B01D02248F8BD204B5A6802F084
S315080093883F025B6813F4800F12D01C4B5968C1F36F
S31508009398881100231B48A1FB0001FEF711FF174B94
S315080093A85B68C3F3014301335B00B0FBF3F0F8BD18
S315080093B8124B5B68C3F388131E4600275C01002519
S315080093C8E41A65EB0705A90141EA9461A001001BA7
S315080093D861EB0501CB0043EA5073C400A01943EBBF
S315080093E807018B0243EA9053840220461946002354
S315080093F8FEF7E6FED3E70348F8BD00BF003802408B
S315080094080024F40040787D01002800F0A28070B599
S315080094180446524B1B6803F00F038B4209D2CBB2A2
S315080094284E4A1370136803F00F03994201D00120BE
S3150800943870BD236813F0020F17D013F0040F04D079
S31508009448474A936843F4E0539360236813F0080F78
S3150800945804D0434A936843F460439360404A936848
S3150800946823F0F003A068034393600D46236813F0BE
S31508009478010F31D06368012B20D0022B25D0384A3A
S31508009488126812F0020F66D035498A6822F003027C
S3150800949813438B60FFF7C2F90646314B9B6803F006
S315080094A80C036268B3EB820F16D0FFF7B7F9801B77
S315080094B841F288339842F0D9032070BD284A1268C9
S315080094C812F4003FE0D1012070BD254A126812F057
S315080094D8007FD9D1012070BD204B1B6803F00F030C
S315080094E89D4209D2EAB21D4B1A701B6803F00F0396
S315080094F89D4201D0012070BD236813F0040F06D0E1
S31508009508174A936823F4E053E1680B43936023688A
S3150800951813F0080F07D0124A936823F460432169A9
S3150800952843EAC1039360FFF71DFF0D4B9B6803F0E1
S31508009538F003F02292FAA2F2B2FA82F2D340094A6A
S31508009548D35CD840084B18600020FFF72FF9002095
S3150800955870BD01207047012070BD00BF003C024065
S3150800956800380240E89D000800000020014B1868F2
S31508009578704700BF0000002008B5FFF7F7FF074B44
S315080095889B6803F4E0534FF4E05292FAA2F2B2FA57
S3150800959882F2D340024AD35CD84008BD003802405C
S315080095A8F89D000808B5FFF7E1FF074B9B6803F429
S315080095B860434FF4604292FAA2F2B2FA82F2D340BA
S315080095C8024AD35CD84008BD00380240F89D000816
S315080095D82DE9F04704460268136923F44053C16825
S315080095E80B4313610168CB6823F4164323F00C0375
S315080095F882680069024360690243E06902431343CB
S31508009608CB602268536923F44073A1690B435361FD
S31508009618E369B3F5004F62D0D4F80080BB4B984590
S3150800962800F01B8103F58063984500F01681FFF763
S31508009638A3FF00EB800000EB80006568AD00B0FB77
S31508009648F5F5B34FA7FB05356D092E01FFF794FF0E
S3150800965800EB800000EB80006568AD00B0FBF5FA0A
S31508009668FFF78AFF00EB800000EB80006568AD0015
S31508009678B0FBF5F5A7FB05356D094FF0640909FB3D
S3150800968815A52D013235A7FB05356D0905F0F00539
S315080096983544FFF771FF00EB800000EB8000666831
S315080096A8B600B0FBF6F6FFF767FF00EB800000EBA5
S315080096B8800063689B00B0FBF3F0A7FB0030400905
S315080096C809FB10694FEA091909F13209A7FB093795
S315080096D8C7F343172F44C8F80870BDE8F087D4F8CD
S315080096E8008003F1804303F5104398455CD003F5E1
S315080096F88063984558D0FFF73FFF00EB800000EBE2
S31508009708800065686D00B0FBF5F5814FA7FB053548
S315080097186D092E01FFF730FF00EB800000EB800093
S3150800972865686D00B0FBF5FAFFF726FF00EB8000C9
S3150800973800EB800065686D00B0FBF5F5A7FB0535FD
S315080097486D094FF0640909FB15A5ED003235A7FB2D
S3150800975805356D096D0005F4F8753544FFF70CFFF6
S3150800976800EB800000EB800066687600B0FBF6F632
S31508009778FFF702FF00EB800000EB800063685B00E0
S31508009788B0FBF3F3A7FB03235B0909FB13694FEA4D
S31508009798C90909F13209A7FB0937C7F342172F4444
S315080097A8C8F80870BDE8F087FFF7FCFE00EB8000F4
S315080097B800EB800065686D00B0FBF5F5544FA7FB14
S315080097C805356D092E01FFF7EDFE00EB800000EB6D
S315080097D8800065686D00B0FBF5FAFFF7E3FE00EB5D
S315080097E8800000EB800065686D00B0FBF5F5A7FB07
S315080097F805356D094FF0640909FB15A5ED003235E5
S31508009808A7FB05356D096D0005F4F8753544FFF7AE
S31508009818C9FE00EB800000EB800066687600B0FBA6
S31508009828F6F6FFF7BFFE00EB800000EB80006368E2
S315080098385B00B0FBF3F3A7FB03235B0909FB13697A
S315080098484FEAC90909F13209A7FB0937C7F34217CD
S315080098582F44C8F80870BDE8F087FFF7A3FE00EBA9
S31508009868800000EB80006568AD00B0FBF5F5284F71
S31508009878A7FB05356D092E01FFF794FE00EB80005E
S3150800988800EB80006568AD00B0FBF5FAFFF78AFEC5
S3150800989800EB800000EB80006568AD00B0FBF5F5CD
S315080098A8A7FB05356D094FF0640909FB15A52D01B8
S315080098B83235A7FB05356D0905F0F0053544FFF780
S315080098C871FE00EB800000EB80006668B600B0FB0E
S315080098D8F6F6FFF767FE00EB800000EB800063688A
S315080098E89B00B0FBF3F3A7FB03235B0909FB13698A
S315080098F84FEA091909F13209A7FB0937C7F34317CC
S315080099082F44C8F80870BDE8F08700BF001001406A
S315080099181F85EB512DE9F04105460F461646984630
S31508009928069C2B681B6837EA03030CBF0123002330
S31508009938B3421ED1B4F1FF3FF3D02CB1FEF76EFF48
S31508009948A0EB08008442ECD22A68D36823F4D073C3
S31508009958D3602A68536923F001035361202385F8E5
S31508009968393085F83A30002385F838300320BDE8C1
S31508009978F0810020BDE8F081704758B310B5044659
S3150800998890F839300BB3242384F839302268D36821
S3150800999823F40053D3602046FFF71AFE226813699A
S315080099A823F4904313612268536923F02A03536109
S315080099B82268D36843F40053D3600020E063202369
S315080099C884F8393084F83A3010BD80F83830FFF713
S315080099D8D3FFD8E7012070472DE9F04182B01E462B
S315080099E890F83A30DBB2202B03D0022002B0BDE84B
S315080099F8F08104460D469046002958D0002A58D0CA
S31508009A0890F83830012B01D10220EFE7012380F8BE
S31508009A1838300023C363222380F83A30FEF7FEFE67
S31508009A280746A4F82C80A4F82E801DE000963B462D
S31508009A38002220212046FFF76DFF00283BD1236925
S31508009A4833B923685B68C3F3080325F8023B0BE0C0
S31508009A5823685B68DBB225F8013B05E023685B6889
S31508009A6803F07F032B700135E38D9BB2C3B1E38DF9
S31508009A789BB2013B9BB2E385A368B3F5805FD5D05B
S31508009A8800963B46002220212046FFF743FFA0B94F
S31508009A982369002BE2D123685B682B700135E3E75D
S31508009AA8202384F83A30002084F838009EE70120FD
S31508009AB89CE701209AE7032098E7032096E7000029
S31508009AC80C4B1A6842F001021A60002199601A685C
S31508009AD822F0847222F480321A60074A5A601A6899
S31508009AE822F480221A60D9604FF00062034B9A600C
S31508009AF8704700BF003802401030002400ED00E02F
S31508009B08014B024A9A60704700ED00E000800008A1
S31508009B1800B593B001230693079302230C934FF4D9
S31508009B2880020D9219220E92F0220F9210930523A5
S31508009B38119306A8FFF76EFA00B1FEE70F23019303
S31508009B4802230293002303934FF4A05304934FF47C
S31508009B5880530593032101A8FFF756FC00B1FEE7D9
S31508009B6813B05DF804FB08B5FFF7CAFFFEF734FE25
S31508009B78FFF7CEFF00F0D2F8FEF7E6FD08BD08B5F8
S31508009B88FFF7F1FFFEF754FDFEF7E8FDFEF7D6FDF1
S31508009B98FAE70000F0B58DB000240194464B5A6CDC
S31508009BA842F480425A645A6C02F480420192019A3D
S31508009BB802941A6B42F002021A631A6B02F0020246
S31508009BC80292029A03941A6B42F008021A631A6BF5
S31508009BD802F008020392039A04941A6B42F02002D0
S31508009BE81A631A6B02F020020492049A05941A6CF6
S31508009BF842F480221A641A6C02F480220592059AA5
S31508009C0806941A6C42F000721A641B6C03F000730F
S31508009C180693069B0320FFF79BF8224621466FF01A
S31508009C280B00FFF7A7F8224621466FF00A00FFF750
S31508009C38A1F8224621466FF00900FFF79BF822464D
S31508009C4821466FF00400FFF795F8224621466FF083
S31508009C580300FFF78FF8224621466FF00100FFF749
S31508009C6889F8224621464FF0FF30FFF783F84FF46C
S31508009C78807307930125089509950A9507A90F483A
S31508009C88FFF7D6F84FF440770797022608960995FE
S31508009C9803250A9507230B9307A90948FFF7C8F868
S31508009CA80797089609940A9509230B9307A905485F
S31508009CB8FFF7BEF80DB0F0BD0038024000140240A8
S31508009CC8000C024000040240DFF834D0002103E00B
S31508009CD80C4B5B58435004310B480C4B42189A42BC
S31508009CE8F6D30B4A02E0002342F8043B094B9A4292
S31508009CF8F9D3FFF7E5FE00F031F8FFF740FF7047A4
S31508009D0800000220109E0008000000200400002021
S31508009D18040000201C010020FEE7000008B5FFF734
S31508009D2825FC084BA3FB00308009FFF755F80420EB
S31508009D38FFF768F8002211464FF0FF30FFF71AF8C8
S31508009D4808BD00BFD34D621008B5FEF767FD08BD0C
S31508009D5808B5FEF75BFDFFF766F808BD70B5002580
S31508009D680C4E0D4CA41BA410A54209D100F01AF8F4
S31508009D7800250A4E0A4CA41BA410A54205D170BD9D
S31508009D8856F8253098470135EEE756F825309847AE
S31508009D980135F2E7089E0008089E0008089E000894
S31508009DA80C9E0008F8B500BFF8BC08BC9E4670476C
S31108009DB8F8B500BFF8BC08BC9E46704712
S31508009DC405020602060307030803090309040A042D
S31508009DD40B040C040C050D050E050F050F061006DD
S31508009DE41007100800000000000000000102030428
S31108009DF40607080900000000010203042D
S30D08009E00F8E3FF7F01000000F2
S30908009E08AD81000812
S30908009E0C8981000832
S30908009E100024F40028
S70508009CD185
